:020000040000FA
:1000000000880002210100001D0100001D01000008
:1000100000000000000000000000000000000000E0
:100020000000000060320000A83200001D01000046
:1000300000000000000000001D0100001D01000084
:100040001D0100001D0100001D0100001D01000038
:100050001D0100001D0100001D0100001D01000028
:100060001D0100001D0100001D0100001D01000018
:100070001D010000510100001D0100001D010000D4
:100080001D0100001D0100001D0100001D010000F8
:100090001D0100001D0100001D0100001D010000E8
:1000A0001D0100001D0100001D0100001D010000D8
:1000B0001D0100001D010000000000000000000004
:1000C0000348854600F018F8004800478101000009
:1000D0000088000203460B439B0703D009E008C9D0
:1000E000121F08C0042AFAD203E00B780370401CE8
:1000F000491C521EF9D27047064C0125064E05E0F8
:10010000E36807CC2B430C3C98471034B442F7D338
:10011000FFF7DAFF3032000040320000FEE7000057
:1001200006480168032291430160016801220A43E5
:10013000026000F005F800F043F8C04628000040D7
:100140000148024901607047008000020026B803A0
:1001500080B582B0002001902B48C268002A02D0EE
:1001600001A80021904702B080BDC0460121814016
:10017000024802688A4302607047C046200000407F
:1001800070B50024204600F01FF80A4D0A4E0B4AB5
:1001900028463146FFF79EFF01204006C022314627
:1001A000FFF798FF286880F3088868688047204632
:1001B00070BDC04600A0020238020000F82F000007
:1001C00000480047C1000000B0B5002801D0012060
:1001D000B0BD032081020C4802680C4B5350002430
:1001E0009460012253030A4D2B60BFF34F8FBFF37E
:1001F0006F8F084D2B6003685A5084720481102061
:10020000FFF7B4FF2046B0BD0480000251E5CC1AD0
:1002100080E100E080E200E002E008C8121F08C1AF
:10022000002AFAD170477047002001E001C1121F77
:10023000002AFBD17047000000FC020279A60202EE
:1002400005A3020205A30202000000000000000056
:1002500000000000000000000000000060CF02026B
:10026000A8CF020205A30202000000000000000067
:1002700005A3020291A80202A7A1020205A302029D
:1002800005A3020299A6020205A3020205A3020227
:100290009DA2020235A3020205A3020205A30202E7
:1002A00005A3020209A3020205A3020235A9020264
:1002B00005A3020205A3020205A3020205A302028E
:1002C00005A30202B9A80202D5A8020205A30202F0
:1002D00005A3020205A30202F5A80202FFA802027A
:1002E000A9A1020205A3020205A3020205A30202BC
:1002F00000000000000000000348854600F040F8C0
:100300000048004769C0020200FC020230B50B46FB
:10031000014600202022012409E00D46D5409D42DF
:1003200005D31D469540491B254695404019154665
:10033000521E002DF1DC30BD03460B439B0703D05A
:1003400009E008C9121F08C0042AFAD203E00B789A
:100350000370401C491C521EF9D27047D2B201E012
:100360000270401C491EFBD270470022F6E710B510
:1003700013460A4604461946FFF7F0FF204610BD13
:10038000064C0125064E05E0E36807CC2B430C3CE8
:1003900098471034B442F7D3FFF7B2FF40CD0202C2
:1003A00060CD020230B58C180278401C13071B0F79
:1003B00001D10378401C120906D10278401C03E0E9
:1003C00005780D70401C491C5B1EF9D101E00B70D3
:1003D000491C521EFBD1A142E6D3002030BD70471C
:1003E0007047B0B5044645180020AC4205D22178CC
:1003F00080B200F0A5FB641CF7E780B20024214620
:1004000000F09EFB214600F09BFBB0BD10B504211F
:100410000A060AD0027852B2D3091B241C405200AB
:1004200062400270491E401CF2E710BDB0B50123C6
:100430000022D4B20355DCB20A555C005C401B06B6
:10044000DD171B232B406340DCB2521C012CF0D182
:100450000178FF228154B0BDF0B500210E4A0B4651
:10046000002B0C4605D030CAED5CFF266E40A45D23
:10047000083A632565400426370606D06700E4B2D3
:10048000E4093C196540761EF6E7C5545B1C01245F
:100490002402A342E4D1F0BDF4E9020270B50022C7
:1004A00013461446E5B2465DB34204D06C1CE5B277
:1004B000A542F7D000E0CC545B1C01242402A342E7
:1004C000EFD170BD0B780370491C401C521E1306FF
:1004D000F8D17047BCB5184C20680568002001A908
:1004E0000870C0B2082825D2012211048140294297
:1004F00009D02268516080002018826A002A16D034
:1005000001A8012112E0130283402B4201D00221F5
:1005100004E082402A420AD0032113462268536035
:10052000800020188268002A01D001A89047019815
:10053000401CD4E7BCBDC0461CE80202FEE7000038
:1005400010B509480168CA6920231343CB610269C9
:10055000032A08D1012293050C689C430C605102C8
:10056000C26E0A43C26610BD84E80202F8B50C48A8
:1005700006460C360068876B0024122C0ED001252D
:10058000A5403D4207D03168002904D02046884765
:10059000034800688563361D641CEEE7F8BDC0465D
:1005A00000E90202F0B585B000900025144E0A2043
:1005B0002C46002821D00290039108463146FFF7CF
:1005C000A5FE07463030009948550195FDB20494C8
:1005D0002543681E2C46844177430A213046FFF7A5
:1005E00095FE0646002D01D0019D6D1C02AB0BCB84
:1005F0001B191C46C91B401EDBE705B0F0BDC046F9
:1006000000CA9A3BFEB50C460546E031102200F0C8
:10061000BBFA0194D0340D27284600F077F8102259
:1006200028460294214600F08BF80020042421067D
:1006300006D0C6B2A81900F011F8641E301DF6E706
:10064000029C103C7F1E3806E6D1284600F05EF87A
:1006500010222846019900F073F8FEBDF0B58BB06A
:100660000446C0780890A0780290277804976578AF
:100670000795254E2046B04760780990A0780690EF
:10068000E078019020780A902046B0473146A07863
:10069000059020780390E07800906678204688479F
:1006A000394669406078A2784240E3785340207828
:1006B00058400246029B5A404A400A9D6A40019FA8
:1006C0007A40009D6E407240E270089A504041406E
:1006D000069D69407940039F059A57407940A17073
:1006E00001465940049A5140099A5140694071406D
:1006F00061700799484058400A99484050407840F6
:1007000020700BB0F0BDC046D5A10202417B427AF9
:100710004273427943784371427241708178827AA0
:10072000827081728179827B82718173C178C27992
:10073000C270C27AC271C27BC173C27270470000BC
:10074000B0B5064B04781C5D0D7865400570491CFA
:10075000401C521E1406F5D1B0BDC0468CEC0202FE
:10076000F0B587B004460120019005902F48202263
:10077000214603782370401C641C521E1306F7D1D7
:1007800040393D3106A80422FFF79CFE3F20C043BC
:10079000049020210294EF2945D86518049C203448
:1007A0001C2008401028039121D0002823D1009557
:1007B00006AD687806992870A878EA78AA706870FB
:1007C000E97004262846314600F070F905AF284646
:1007D000009D3946324600F0D7F9019A50B2C0095F
:1007E0001B21014052004A4001923A7003E006A8E2
:1007F000042100F05BF904982F462D1806AE042260
:100800003046294600F0C0F9069838557078212105
:100810006854B07822216854F078232168540399F1
:10082000091D029CB7E707B0F0BDC046CCCC020260
:10083000F8B500F071F800281FD16C4611482080EF
:1008400001273A030025104E2846314600F0F2FFFA
:100850001036022328463146224601F069FB7C0609
:100860001920020309492046FFF766FD206880F33E
:100870000888606800198047F8BD0A2000F066FD0E
:1008800000F004FBFFFF000000D0020400A0000401
:1008900070B505464E1C0024761E05D0284600F093
:1008A00087F80128F7D100E0E443204670BD00003E
:1008B00006480168032291430160016801220A434E
:1008C000026000F00DF901F053FEC0462800004020
:1008D00080B50B490868002800D480BD094802682B
:1008E0000423032A01D01A4300E01A460A6006498D
:1008F0000A68002AF1D041680020904780BDC046B8
:100900002C10014000E80202F4F1020280B500F070
:100910005BF8002080BD0000FEB568460026068119
:10092000019600963320FFF7F1FF114800F038F9E7
:100930000446012812DB0F480F4FB8470F48B8474D
:100940006D4628462146FFF72DFE0DA0B8472846E4
:10095000B8470EA0B84710A0B84706E00220C04331
:10096000844201D3664200E00426F0B2FEBDC046D8
:1009700010F20202ECCC0202B5A702028CEA0202DB
:100980000A0D2053697A653A2000000020427974EC
:1009900065730D0A000000002D2D2D2D2D2D2D2D00
:1009A0002D2D2D2D2D2D2D2D2D2D2D0A000000004E
:1009B0000D49896C4A69D20501D400207047496805
:1009C000017001207047C046E0B501A908700648D3
:1009D000806C416A0029FCD101A901200023024654
:1009E00002F036F88CBDC04654E9020210B5044648
:1009F0002078002803D0FFF7E7FF641CF8E710BD5C
:100A000070B50278302A27D1427820231343782BFF
:100A100022D18278002A47D05622D34300240222D2
:100A20000B2A41D0855C002D31D02E46413E062E4A
:100A300002D21E4620360AE02E46613E062E1E4693
:100A400005D32E46303E092E1FD81E46273675196F
:100A500024012C19521CE3E7002213460B2A23D051
:100A6000845C002C1CD04B2C17D04D2C11D06D2C3D
:100A70000FD06B2C11D02546303D092D05D80A2505
:100A80005D432B19303B521CE8E700200AE00C6064
:100A900007E0002A08D01B0502E0002A04D09B02D0
:100AA0000B6001200B2A00D3002070BD10B5054A51
:100AB00003789468E35C0370401C491E0B06F7D171
:100AC00010BDC046F4E9020280B504480168491C23
:100AD00001600069002800D0804780BDF8F1020263
:100AE00001480249016070470CE802020026B80381
:100AF000E0B50D4908680022C2600192CA68002A68
:100B000002D0016801A890478CBDC046E0B50649F7
:100B100008690022C26001220192CA69002A02D03B
:100B2000016801A890478CBD64E8020280B50020EE
:100B300001F02AFE80BD80B5012001F025FE80BDB8
:100B4000B0B501231A028A18D903074B44001506D1
:100B5000ED0F2C19084200D05C40204654000A4298
:100B60002246F3D080B2B0BD21100000E0B50020D5
:100B700001900448C268002A02D001A800219047D1
:100B80008CBDC046E4E9020210B50B7804785C40E5
:100B90000470491C401C521E1306F6D110BD000003
:100BA000F0B585B0044600F089F9B24D0027022067
:100BB0000090A8806F80B048E8602F616F61AF61DE
:100BC00001200190000504900394EF612F626C6294
:100BD000384602F0A1F8AF6228460499FFF758FEA4
:100BE000002810D06869A969012901DB401C6861EF
:100BF000062800DB04E14320FFF7E6FE039C286A99
:100C00000028E5D0F8E0287801280CD002289B4A7B
:100C10000CD0042840D0182865D0412800D1F7E036
:100C20006128DFD1F4E08026944A01E001998E0228
:100C30001070052434430120E88080B28F4984423B
:100C400008D908180499FFF723FE0028CAD1E888BC
:100C5000401CF1E78878FF2242404978914200D059
:100C6000D6E06888884203D02978012900D0CFE0F7
:100C7000401C6880814CE01C3146FFF7B2FB042128
:100C80003143615C03223243A25C1202511881425B
:100C900000D0BDE0AE6200E0AE6A00246C61002EC0
:100CA00000D1A3E0701C00D1CFE074484178E8691E
:100CB000C2B2914223D1002845D0686A6F49C91C4D
:100CC0003246FFF739FB03986863AC63AB6A9C421A
:100CD00017DA2946443100F00DF9686B103068636B
:100CE000AC6B1034F1E728460499FFF7D1FD0028DA
:100CF00000D077E72878182800D073E79FE0152008
:100D00007AE7688880025E494018039AEA6328649B
:100D1000E9680026304601F00BF9002800D083E096
:100D2000296CE868884202D0AA6891427CD9A96AF5
:100D30000818E8600620FFF747FE52480660A888BA
:100D4000401CA8804CE04D4BD87800287FD0002074
:100D5000D91CE862296301991A1800290AD0FF28D2
:100D600008D8D178484C2154401C111DE8622963F1
:100D70001179F1E70021444B1954101DE9622863F1
:100D8000009AD2430292425C202A0FD00E290DD83D
:100D900042186B18521C029CA418A4783E46542793
:100DA000DC553746491CE9622A63ECE72846543093
:100DB00000224254491CE96229460831FFF720FE0F
:100DC00019200203501CA968814248DC00202A49EE
:100DD00000F030FD0620FFF7F7FD4320FFF7F4FD9C
:100DE0000198A861E869401CE86107E70620FFF761
:100DF000EBFD01202862039C286900282DD1E4E640
:100E000018252846FFF7E0FD2846FFF7DDFD08E03E
:100E100018242046FFF7D8FD2046FFF7D5FD00989F
:100E2000C743384605B0F0BD18242046FFF7CCFD77
:100E30002046FFF7C9FD0098C043471CF1E700209A
:100E400068610098C043801CA8620620DDE7062088
:100E5000FFF7BAFD012028612862AF68E1E7182496
:100E60002046FFF7B1FD2046FFF7AEFD0298871C34
:100E7000D7E7C04608EA020200A00004ECED020237
:100E8000009C000410F702028CEA0202BFF34F8FAD
:100E9000084809490160BFF34F8F00BFFDE7C04616
:100EA000BFF34F8F034804490160BFF34F8F00BF6A
:100EB000FDE7C0460CED00E00400FA0570B51C4EDD
:100EC0000A4C0B4D3560746028462146FFF7AEFA98
:100ED0001648B060FFF7C0FAF5602846FFF740FCFF
:100EE0003461B0682146FFF7D9FA70BD8CEC02027C
:100EF0008CEB0202F8B50C460746FFF7DFFF0B4DFF
:100F00001026284639463246FFF7DCFA0848C16801
:100F10003846FFF777FB384621463246FFF734FE66
:100F2000204629463246FFF7CDFAF8BD10F60202F8
:100F3000F4E9020270470000F8B516484C21016040
:100F4000FF240234144F2046B847322000F005FA3F
:100F500000F0DCF80125284600F0E2F8284600F011
:100F600033F800F0CDF80D48B8470026304631463A
:100F700000F09EF92846314600F09AF93046B8470D
:100F80000220B8474734204601F0F6FA01F010FB82
:100F9000F8BDC04648000040F9AE02020102000060
:100FA00070470000B0B505200424064D2146A8472F
:100FB00006202146A84701202146A8470E202146A9
:100FC000A847B0BD19C0020202490A680240824225
:100FD000FBD1704704600040B0B53C4801688A0707
:100FE0003B4C07D501797F221140E369934359189F
:100FF000E1610168890407D55E21405C7F210840DA
:10100000226A8A4310182062172000F0F7F831484E
:10101000016802220A4301218A4302602E482F49B7
:1010200001602F480021C17181791F2529408171FC
:10103000817A427C837C1B029A18C37C1B04D218E1
:10104000037D1B06D218274B9A4218D1427B837B23
:101050001B029A18C37B1B04D218037C1B06D218F0
:10106000214B9A420BD1C27A037B491E122906D822
:10107000190289181D4A914201D12021017201787B
:10108000CA0602D110221143017020682021884332
:10109000206026481649016041680029FCD501F00E
:1010A00053FA0A21C841032800D8FEE71148C16855
:1010B0000F229143C16001680F4A0A400260192063
:1010C00000010E4948600D60B0BDC0468CED0202C3
:1010D0002C000040040200400C060040AF6B100AD8
:1010E0006B0001404D383650312E32360734000047
:1010F000FE1C0080C8600040FEFFC3FF0C040040DF
:1011000080B5172000F072F8002080BD10B51724BC
:10111000204600F073F8204601F01CFA002010BDB4
:101120000121C90701430148016070470060004088
:10113000B0B5C2B2000AC1B2022A0CD0012A12D044
:10114000002A2CD18A1E3148022A19D201220329F1
:1011500026D0510425E02D48426800291BD00146C5
:1011600020390A431AE0294C2568C81E02280ED3EC
:10117000012926D000292DD101208007854330E0A8
:10118000002914D10121490702688A4317E0042984
:101190001DD002201CE0012189078A434260B0BDB6
:1011A000110403221204C36A93435918C1620E4901
:1011B0000A689207FCD50121490702680A430260C8
:1011C000B0BD0520000785432046203808E00120F7
:1011D00000F09EF8044801684906FCD50520000788
:1011E00005432560B0BDC0462C020040012181406E
:1011F000064802688A4302607047C0460121814068
:10120000024802680A4302607047C046200000405E
:1012100080B500F03BF83D4909688900890FC84056
:1012200080BDC04680B5FFF7F3FF38490968090162
:10123000890FC84080BDC04610B505280AD8C046F1
:10124000784400794000874402070F0A121700F023
:101250001DF810BD002010BDFFF7DAFF10BD012002
:1012600081074A6A520004D5FFF7DCFF10BD012058
:101270008107096AC00310BD0120840700F006F849
:10128000616A0903890FC84010BD00000121880769
:10129000026A006AC00001D5044800E0024852001A
:1012A00000D4C8037047C046006CDC020026B803B7
:1012B000042829D8154AC04678440079400087445C
:1012C000020910171E0003200007136883438807D4
:1012D000800812E003208006136883438807000912
:1012E0000BE003208004136883438807000B04E0AD
:1012F000FF200002136883430802181803E01068F7
:10130000FF239843401810607047C04624000040F7
:1013100009490A68094B134000041843086008484B
:10132000002101600749084A0A600D21490242680C
:101330000A4342607047C0464800004080FFFCFFFF
:101340001002004004010040FF0F000080B57D2125
:10135000C900484300F001F880BD00280AD030B42D
:1013600007252C02CD256419604340091238001F5F
:10137000FDD830BC70470000F8B505460120072DA8
:1013800066D80C46002963D0444F38680169C90704
:1013900036D105263046FFF731FF304601F0DAF846
:1013A00003CF0369012213430361002918D40320EA
:1013B0000B4683436D481E588807C00EFF278740A1
:1013C000BE4340278740374368481F501F200840CE
:1013D00082406748026067480260304800680FE05A
:1013E0008A07D20EFF2696400F230B40083B0321AD
:1013F0008B435D495F58B743402696403E435E505D
:1014000069014018012109024218E369DB069B0CBF
:10141000A569ED00EDB2EB18536062685207520BFC
:1014200023685B075B099A18A3685B079B0CD218BB
:10143000E3685B075B0DD21823695B01DBB2D2184E
:1014400063699B07DB0ED2188023134343500020AF
:10145000F8BDC046F8B505460835104C2668F66854
:10146000EE40F50701D00220F8BD069D8600A619C2
:10147000B560400124682018009301231D0246191D
:1014800077680724A7437760F16032610099B16003
:101490004159194341510020F8BDC0461CE80202E1
:1014A00000013A49085840687047C046F8B50546FB
:1014B0000120012D45D80C46002942D0002D03D033
:1014C000012D04D10F2000E00E20FFF797FE290127
:1014D0002E4843580020D86027686568A668F6073C
:1014E000B60FAD072D0FAE192569EA07920EB61893
:1014F000022F04D0012F03D10122164300E0403611
:101500009E60E2681A60214A51188D606269CA6063
:101510004968002916D403220B469343134A9C586A
:101520008D07ED0EFF26AE40B4438026AE40264325
:101530009E501F220A40012191400D4A11600D4A20
:101540001160F8BD8A07D20EFF2494400F230B4090
:10155000083B03218B4304495D58A54380249440F4
:101560002C435C50F8BDC0461CED00E000E400E0F8
:1015700080E200E000E100E00001044A1058016050
:10158000816880220A4382607047C04664E8020294
:10159000F8B50E460446032100F0FAFB0546002884
:1015A00038D1204600F09EFB0621204600F044FC86
:1015B0007C206043EC490F183A6A5643BA69B21866
:1015C00008588260172179563E461736002909D5FA
:1015D000C16920220A43C2610121F96689050268B6
:1015E0000A4302600521204600F026FC307840B214
:1015F00000280FD4084800687D26F100FEF786FE1B
:1016000071014143204600F0E7FB204600F07AFCE0
:10161000012038612846F8BD0CF20202FEB50646EC
:1016200002907C207043D0490F18FD6EECB2601E12
:1016300002280BD228040121000E28D03046019147
:1016400000F040FB0199C00705D020E0032C1BD11E
:101650002804000E1AD038466C302D0C0021019160
:101660000160304600F04EFCE9B20120002902D0B2
:10167000032900D0062038613A6F002A02D002A860
:1016800021469047019902E0002100E0012108462F
:10169000FEBDC046F8B50C460078B34DE9688142FE
:1016A0002BD1032C52D1686EA96E88424ED90024EA
:1016B0000621204600F0C0FB2868E96D81602046C5
:1016C000214600F0B9FB2E4660364CCEE86829680A
:1016D000AC8C264F00979B1BA34200D81C46A30846
:1016E0001431FFF7B7FEA86E0019A866286E00191E
:1016F0002866E86D0019E865F8BDA968814224D123
:10170000032C26D1E88CE96D0918E965296E0918C2
:101710002966A96E0818A866696E814219D9002445
:101720000621204600F088FB2868E96D81600121D0
:10173000204600F081FB296EA868EB8C2A680B4CD0
:10174000009414329B08FFF785FEF8BD002000F0DE
:10175000C9FA0120C1072A6813688B431360E96E38
:1017600022040A4300021043E866F8BD5DB4020299
:10177000BCB50078F24DAA68824237D1032929D13D
:10178000686DA866AA6DAB6A1B18EA652B66AA6C21
:10179000521CAA646A6E82421CD9012000025E308B
:1017A000FFF7DBFD686CA96C022920D381421ED1B2
:1017B000E88C696D0818686500240621204600F051
:1017C0003BFB2868E96D8160296D204600F000FD33
:1017D0002B6D24E00120C2072B681C6894431C6019
:1017E000EA6E0904114300020843E866BCBD022901
:1017F000FCD38142FAD2E88C696D09186965A96D3C
:101800000818A86500240621204600F015FB28686A
:10181000E96D8160E98C204600F0DAFCEB8C296EE2
:10182000A8682A68024C00941432FFF713FEBCBD6E
:1018300039B50202F0B587B004460127880E6AD098
:101840001546002A67D00E468120C004401B8842FE
:1018500061D37C206043BA4908180590818C3046DA
:101860000691FEF753FD002955D128460699FEF74B
:101870004DFD00294FD105988069361A30460699EA
:10188000FEF744FD0746039670190190069E314607
:10189000FEF73CFD0546C01B04900598006A0290C7
:1018A0003146FEF733FD049981420CD2AF4231D26A
:1018B0002046394600F024FA2046FFF7AFFE002804
:1018C000FAD17F1CF2E705900398029E3146FEF79D
:1018D0001DFD0546304668430399081A01983146B4
:1018E00000D06D1C059E6E43FEF710FD049002991A
:1018F00041430198401A03900699B7420ED2204600
:10190000394600F0FDF92046FFF788FE0028FAD19D
:101910007F1CF1E70027384607B0F0BD0398FEF7BB
:10192000F5FC0646049FBD420AD220462946FFF731
:101930002FFE2046FFF772FE0028FAD16D1CF2E759
:1019400005987843059000273D46B542E3D20598B7
:101950002918204600F0D4F92046FFF75FFE002842
:10196000FAD16D1CF1E7C04684E80202F8B5002800
:1019700001D00124B0E07826E04FB85D002801D006
:101980000024A9E0002904D0384614301422FEF7C0
:10199000D3FC0024FC6615252846FFF72FFC2846BB
:1019A00000F0D8FD204600F09DF9B88AB97D0907FE
:1019B000090B0918F87DC207D20889188207D20FCF
:1019C00052058918C206D20FD20589184207D20FD4
:1019D000D20689188206D20F520789180007C00F55
:1019E00080070843396808600A21204600F024FA7D
:1019F0003220FFF7B2FC0821204600F01DFA20211A
:101A00002046224600F0FCF93868017D0A46C23AB9
:101A1000534253417422BB54027D007DC22903D13D
:101A2000F97D0120084014E000240321204600F045
:101A300003FA20212046224600F0E2F93868007DB2
:101A4000420801201040F97D0A43D20701D001402D
:101A500004D001214140002000F07EFB7720385C5B
:101A6000012803D102200021FFF722FC0024204698
:101A700000F048FA1720385600282AD57868002840
:101A800017D4032102468A43154953588507ED0EA2
:101A9000FF21A9408B438021A9401943104BD1500D
:101AA0001F210140012088400E4908600E4908604E
:101AB0000FE08107C90EFF238B400F220240083A36
:101AC00003208243054815589D4380238B402B43B8
:101AD00013500120B85538612046F8BD1CED00E0D8
:101AE00000E400E080E200E000E100E0FEB51E4618
:101AF0001746029105460621019100F09DF97C24CC
:101B00006C43CC48005902998160029528463146C1
:101B100000F05EFBC7480019002E05D03978026836
:101B200011757F1C761EF7E7984800687D21C90073
:101B3000FEF7ECFB01994143029800F04DF9FEBD20
:101B400084E80202F0B58FB004460126880E00D169
:101B5000B0E01D46002B00D1ACE00F46049281207E
:101B6000C004401B884200D2A4E00221204600F0BD
:101B70000FF90646002800D09CE00397204600F0AD
:101B8000B1F87C206043E8490F18F87D40060295C3
:101B900028D4069428463D462435B98C0191FEF799
:101BA000B5FB059000240598844257D2062106987B
:101BB00000F042F92888604303994018396888602A
:101BC00000260698314600F037F9049A28888642A4
:101BD00006D2604310183968097D8155761CF5E7F7
:101BE000641CE0E7032000260399F96504993A464E
:101BF000603262C2F8660120C00739680A68024391
:101C00000A600621204600F017F9386803998160C0
:101C10002046314600F010F907AD28492022284619
:101C2000FEF78AFBBC8CF8682946029DFFF7A4FBEF
:101C3000F8683968224A0092AC4200D32C46A308C7
:101C40001431049AFFF706FCB86E0019B866386EB6
:101C500000193866F86D0019F8652BE005980199B0
:101C600041430298441A1BD00621069800F0E4F87C
:101C700028880599484303994018396888600026E8
:101C80000698314600F0D8F8049AA64208D228886F
:101C90000599484380193968097D1154761CF4E789
:101CA000069C204600F01EF8204600F02BF901208B
:101CB0003861002630460FB0F0BDC046B0CB0202FE
:101CC0005DB4020210B50446022100F0B5F82021EF
:101CD0000022204600F094F87C2060439249085886
:101CE000007D10BD80B57C2141438F4A52581021A0
:101CF000D1610A4600F084F880BDC04684E8020243
:101D0000F8B50E460446032100F042F805460028C7
:101D100039D12046FFF7E6FF0621204600F08CF877
:101D20007C20604380490F18BA8C5643BA69B218B8
:101D300008588260172179563E461736002909D582
:101D4000C16920220A43C2610121F966890502683E
:101D50000A4302600421204600F06EF8307840B259
:101D6000002810D4094800687D21C900FEF7CEFA8A
:101D70004B21C9004143204600F02EF8204600F0D8
:101D8000C1F8012038612846F8BDC0460CF20202B5
:101D900070B50123EFF310821A4002D1EFF31084E3
:101DA00072B67C244443E948041926690020062EB3
:101DB0000DD81D46B540EE06760F04D1612635429A
:101DC00003D0184603E0022001E010342160002A0D
:101DD00000D162B670BDC04670B50C46054600F035
:101DE000E1FB06462846FFF76DFFC00707D06420D9
:101DF000FFF7B3FA00F0D6FB801BA042F2D970BD0A
:101E0000F8B500920D467C214143EF48441827461F
:101E1000143700F0C7FB06462068C06928400099C7
:101E2000884205D100F0BEFB801B39888842F3D977
:101E3000F8BDC04684E80202F0B587B00D460446FE
:101E400001210A46FFF7DCFF0227204639463A46C1
:101E5000FFF7D6FF142303956B43DC20604328492A
:101E600008180590C018068A8568C17C06917C21F7
:101E700004946143EE4A52187424145D012C12D16B
:101E800002970196039E012E00D00295012EE84F85
:101E900001D1382406947524125D012A019C029D0B
:101EA00004D0224603E03246E14F03E00322072E2E
:101EB00000D02246069EDF4C14403606AD07ED0AE0
:101EC000AD192C19059DEB58DB075B0CE418436832
:101ED000DD072D0C6419857C6D076D0B6419C068D6
:101EE0004007000A201879584860002A06D0012BC4
:101EF00004D1022100220498FFF782FF07B0F0BD51
:101F0000F0CB020210B5044601210A46FFF778FF24
:101F1000022120460A46FFF773FF7C206043C44934
:101F200008580249816110BD84E80202000093EB69
:101F3000F0B593B005460127880E00D102E11E4698
:101F4000002B00D1FEE00C460A928120C004801BC9
:101F5000884200D2F6E004212846FFF719FF074621
:101F6000002800D0EEE07C2009956843B04902903B
:101F70000F18BC65002107917965701E0690001945
:101F8000B964B9690391621A0A99B962FC6238634B
:101F9000104605927A63F98C0891FEF7B7F9054669
:101FA000B8630698059908180899FEF7AFF90695E1
:101FB000411B4A1C3B463C3307C3079A0029314664
:101FC0000AD0089D68433119039BC91A0A1A069959
:101FD0006943181B401941183D464835384658306A
:101FE00006903C465434F9643A650998FFF77AFE46
:101FF00039464C31F87D40060497079150D43E464F
:1020000044363946403108913946263103915037DC
:1020100005970120069F029628603368984200D9F0
:1020200089E008990968012907D000290ED12068A4
:102030000A990A183968079823E0012808D09842BD
:1020400023D120680A990A18396819E0012811D1AA
:1020500020680A990A183968079F3B680998FFF7B2
:1020600045FD3868069F39680918396021680818E5
:1020700020600AE021680A9A52183968984207D10C
:10208000059803680998FFF731FD2868401CC3E7ED
:10209000039E33880998FFF729FD3088029EE2E706
:1020A0000BA80A902A492022FEF746F902986049B7
:1020B000085801680122D2070A430260B8680A99E9
:1020C000FFF75AF902200A900027069B1968049826
:1020D000826AC1650266466687660A99C166079E7E
:1020E000306821680918216029684A1C2A601A682A
:1020F00010181860002925D1049D294660310A91E5
:102100002E465C362C46083406210998FFF794FECB
:10211000286831688160079E3168099800F058F896
:1021200033680A98016820682A680A4C00941432BF
:10213000FFF790F906E00998FFF7E4FE0120049903
:1021400008610027384613B0F0BDC04684E802029B
:1021500070CB020239B50202B0B50D460446062125
:10216000FFF76AFE07212046FFF766FE7C206043EA
:102170002F4909187420085C012811D1681E854177
:10218000AA01086802750022027575228A5C012A7C
:102190000ED114307622895C4A424A41510006E051
:1021A000086800210175691E8D41690014300170B5
:1021B000064800687D21C900FEF7A8F828214143A0
:1021C0002046FFF709FEB0BD84E802020CF20202CD
:1021D00070B50D460446012631463246FFF710FE23
:1021E000022120460A46FFF70BFE7C20604310497F
:1021F0000A187423D25C012A01D0F30400E03305ED
:102200000C4E2E40F318012A02D01922520601E08A
:102210000722D2069A18084BD21808584260002D9F
:1022200004D0022100222046FFF7EAFD70BDC0461F
:1022300084E80202FF3F00000080800010B5012406
:102240002046FEF7DBFF204600F084F9002010BD99
:10225000124A072809D880000F2383408140194083
:10226000106898430843106070470F280AD8800010
:1022700020380F2383408140194050689843084319
:1022800050607047800040380F23834081401940E0
:1022900090689843084390607047C04634000040FF
:1022A0008AB0FEF749FEFEF77DFEFEF795FE00249C
:1022B000204600F0C1FC7249204600F0DFFCFFF729
:1022C000BDFFFEF76DFE02AE6E4920223046FEF7DE
:1022D00033F820462146FFF749FB012420463146CA
:1022E00000F00EFB68A0FEF781FBC820FFF72EF878
:1022F000009466066C4D0024204600F00DFD01AAF6
:102300006B481080694F1037022320463946FFF78B
:1023100019FC0020FFF782F90028FAD101A80088F3
:102320006449488064498842009C0BD063498842D4
:102330001CD05F49884255D17FA0FEF757FBFEF7BE
:1023400077FA61E05EA0FEF751FB204600F07AF9D3
:102350007D20C000FEF7FAFF1920020330465D49D8
:10236000FDF7EAFF306880F308884AE05AA0FEF7DC
:102370003DFB5FA0FEF73AFBFEF7A0FD2203002421
:1023800020464A49FFF756FA01AD02232046494C40
:1023900039462A46FFF7D6FB2888434D2080474917
:1023A000884211D1009800F04DF9C820FEF7CEFF09
:1023B0001920020330462946FDF7BEFF306880F33E
:1023C00008887068801980474DA0FEF70FFB192020
:1023D0000203002738462946FFF72CFAA0600028A0
:1023E00016D011E0204600F02DF9C820FEF7AEFF10
:1023F0001920020330462946FDF79EFF306880F31E
:102400000888706880198047C820FEF79FFF72E730
:102410004048A080464E474DE76080B2874223DAAD
:10242000F801811980222846FDF786FF00247F2CC1
:1024300006D828191F491031FEF75CFD1034F6E765
:102440001C4FF868C0011849411800248023204619
:102450002A46FFF76DFDB86020463C4600F05CFC64
:10246000B888F9684F1CD7E70A20FEF76FFF2AA04B
:10247000FEF7BCFA7D208000FEF768FFFEF710FD36
:1024800010E80202D0CB02024D4B383030302D42E2
:102490006F6F744C6F616465722D56312E31C6F4C6
:1024A000B6AF0D0A0000000000A0000400D0020436
:1024B000AAAA00006CEA0202CCCC0000BBBB000060
:1024C000BDF8C8EB4F54412CC9FDBCB6C6F4B6AF3D
:1024D0000D0A0000004005044F5441CDEAB3C92C59
:1024E000BDE2C3DCCEC4BCFEC6F4B6AF0D0A00002C
:1024F0004F5441B9CCBCFEBDE2D1B90D0A00000079
:10250000B2C1B3FDB1EAD7A2CEBBB3C9B9A60D0A19
:1025100000000000210300004F5441BDE2C3DCB3C2
:10252000C9B9A6A3ACD7BCB1B8D6D8C6F40D0A00B9
:1025300000F0020414F70202B4AEBFDAC9FDBCB663
:10254000C6F4B6AF0D0A0000014800687047C046E7
:102550000C00004001218140044A1F2802D010686D
:102560008843106010680843106070471C000040EA
:1025700000480047C1A0020210B5401E074948604C
:10258000FF200006064A13688343032084071B19B3
:10259000136000228A60086010BDC04610E000E0B1
:1025A00020ED00E080B50020FEF77AFF404280BDBC
:1025B000B0B586B06C460F4918222046FDF7BCFE28
:1025C000002528462146FEF771FF03992846FEF7AD
:1025D000D3FF0198012801D0082400E0042400283A
:1025E00000D104460220FEF727FEE04002490860C1
:1025F00006B0B0BD2CCB02020CF20202F8B50446C4
:102600000325002801D0284600E004204D430C4E4D
:102610007719B978FEF74CFE48206043B74909584E
:10262000CA68802310461843C860705D7C78240215
:102630002018C8629A43CA60FEF78FFEF8BDC046F4
:1026400044CB020270B5012801D9012070BD482297
:102650004243FB4B9C58A5691F218D43A56106256C
:10266000A5600F2525629C18A27C002A05D1627CFA
:10267000002A02D1227C002A14D06368002B11D4D6
:10268000251D0B40012216469E400C4B1E60BFF3D9
:102690004F8FBFF36F8F2B68002B03D40B409A40F2
:1026A000EA490A60002803D0012804D1092000E08B
:1026B0000820FEF79BFD0020A06170BD80E100E0D6
:1026C000F8B50C460078DE4EF168814209D0726D93
:1026D000824206D0B168814212D0326D82420FD060
:1026E000F8BD0D1A681E85410095482068433018D2
:1026F000032C15D1876B1021284600F053FA19E0FE
:102700000D1A681E85410095482068433018032C37
:1027100019D1C169002921D01C3000210160F8BD08
:1027200081691830302902D00168102901D1802137
:10273000016000274820684330180021816301624E
:102740008162243017E081691830302902D0016895
:10275000202901D180210160002704E0C76B2021DE
:10276000284600F01FFA4820684330180021C16352
:10277000C1624163303000210160002FB0D0684653
:102780002146B847F8BDC046FEB50290482215461E
:102790004543AB494B59DE690F2434404E19357C13
:1027A000002D1FD04F2149025A690A4249D0996928
:1027B0000422914399610221196201218907641859
:1027C000F461F56B202100F0EDF90020F063F06278
:1027D0007063303600203060002D36D002A82146CC
:1027E000A847FEBD0C2C30D87C4424796400A74453
:1027F000432C452C062C7F812C2C2C2C0600B369F5
:10280000202B03D018363368302B1ED104461046D7
:10281000134601946343CD182C6B2F4634376E6BEF
:10282000A6420A4612D2D658716909070ED57468B5
:1028300039684B1C3B60EB6A5C54029C11460246B3
:10284000E5E70C2CB3D0012CB1D0FEBD3968A14214
:10285000FBD12E463036D1588A6905239A438A61C6
:10286000E86B00902021019800F09CF90024EC63B3
:10287000EC62009D3C60ADE701203CE008241C6256
:10288000B469102C04D0344618342468302CDCD1C0
:10289000746AB56AA54213D13546243537462837C0
:1028A0009969022291439961B16B0091102100F066
:1028B00079F90024B46334623C602E46009D89E7B8
:1028C00050430B189D6AA542BFD20646085844697A
:1028D000A407BAD51C46283425686E1C26601B6ADE
:1028E0005B5D0360029813464343CB185C6AE7E7DD
:1028F000022000E004201862FEBDC04654E9020236
:10290000FEB50E460546022803D3002E01D1012450
:1029100094E0002D03D0012D08D1092400E0082403
:102920002046FEF76BFC2046FFF714FE4821029577
:102930006943C04A505883691F240194A3438361AB
:10294000062383600F230093036257180024BC62A0
:10295000BC63FC633C627C62FC623C63317F397423
:10296000727F7A74B27FBA747C637368B268F568F8
:1029700092002A435B1E032B0ED8C0467B441B7972
:102980005B009F4401030507082304E0182302E0CD
:10299000282300E038231A433D461235C260C90798
:1029A000090F72699201D2B28918B2699207920E28
:1029B0008918491C816079613169012901D122217D
:1029C000016131680298FFF719FE2878002809D1C3
:1029D000384611300078002804D13846103000788D
:1029E000002829D07868002816D4032102468A439B
:1029F000154953588507ED0EFF26AE40B343802698
:102A0000AE401E4356500199014001208840C04904
:102A10000860C04908600FE08107C90EFF228A40A4
:102A2000009D0540083D0320854306482B589343ED
:102A300080228A401A432A500120B8612046FEBDF8
:102A400054E902021CED00E000E400E080E200E056
:102A5000F0B58DB005460C900120002900D19DE015
:102A60001646002A00D199E01C460F461021284640
:102A700000F0B2F8002800D090E0482318466843E0
:102A80006C4922460C1800210291A162A2632762C0
:102A90006662217C0029039308D004A814210190C8
:102AA000FDF763FC012D1DD018201CE0A17C00293E
:102AB00036D0604F5D43785979198A6AB2422AD27A
:102AC0004269920727D50A46283213685C1C1460B5
:102AD000096AC95C039B01600C9D1846684338185D
:102AE000466AE7E71A200B90029D0A95022009909A
:102AF000E0680199FEF740FC0C98039941434D486A
:102B000042584018C0682649009139463346FEF7BE
:102B1000A1FC284642E0816982220A4382613CE0AE
:102B20004449085881690A0602D58022914381618F
:102B3000002702973F4A1946694350585418A16A22
:102B4000B1421DD247694F2149020F4212D141695A
:102B5000890709D5214628310A68531C0B60039B5D
:102B6000216A895C01600C9D18466843314A10183F
:102B7000466AE0E7022101620121029189070F43C1
:102B8000416A0029FCD11021284600F00BF8A26B05
:102B9000002A02D00CA83946904702980DB0F0BD2B
:102BA00089C4020210B50123EFF310821A4002D14A
:102BB000EFF3108472B6482444431E480019846918
:102BC0008C4384618169002901D118300360002A97
:102BD00000D162B610BDC046B0B502460120EFF389
:102BE0001083034002D1EFF3108472B6482454439B
:102BF000104A12199569002D18D0802D16D0183260
:102C00000024102D09D0202D0BD0302D07D0402DC1
:102C10000CD0012D09D1116007E0202903D002203A
:102C200004E01029FBD1302010602046002B00D199
:102C300062B6B0BD54E90202B0B5002801D001244B
:102C400018E0032081023D4802683D4B53500024A8
:102C5000946001225303084D2B60BFF34F8FBFF3E5
:102C60006F8F2B4D2B6003685A50847204811020A3
:102C7000FEF7BCFA2046B0BD80E100E0F8B50C4696
:102C800001460120002902D0002C00D1F8BD637953
:102C9000227915461D43F9D00F012848C619B37291
:102CA0007272A068F06010252846FEF7A7FA284641
:102CB000FFF750FC2148C2590320810220485050A0
:102CC000206810600020D06033460A33747A002CEC
:102CD00003D094680225254395601B78002B0ED005
:102CE000FF221202094B1C6894430122D503641988
:102CF0001C605203064B1A60064B1A6032689368D8
:102D000001242343936054503472F8BD0CE400E076
:102D100080E200E000E100E00146012000290CD142
:102D200006490A7A002A08D003208202096804486A
:102D300088500020C86001238B507047E4E90202EC
:102D400051E5CC1A02E008C8121F08C1002AFAD1C6
:102D500070477047002001E001C1121F002AFBD11B
:102D600070470000000000000000000001000000AB
:102D7000FFFFFFFF000000000000000059062014C4
:102D8000032145012882003241003219004113001D
:102D9000390300B506002D03002D02002201002298
:102DA00001003E01002000000000000000000000C3
:102DB0000000000000000000000000000200000011
:102DC00000000000140000000200000007000000E6
:102DD00002000000020000000000000002000000ED
:102DE00000000000140000000200000001000000CC
:102DF00002000000020000000200000000000000CD
:102E000014000000000000000700000000000000A7
:102E100000000000030000000000000000000000AF
:102E200000000000010000000000000000000000A1
:102E30000200000004000000001003EB000000008E
:102E40000100000001000000040000000001003249
:102E50000000000000000000000000000100000071
:102E6000010000050000000000000000000000005C
:102E7000010000000100003500000000010000001A
:102E8000000000000400000000000020000000001E
:102E9000010000000000000004000000000000D855
:102EA0000000000001000000000000000100000020
:102EB000000000060000000001000000000000000B
:102EC00001000000020000010000000000000000FE
:102ED00000000000010000000300009F000000004F
:102EE000010000000000000001000000000000B927
:102EF00000000000010000000000000001000000D0
:102F0000000000AB210504198912130018DECA0164
:102F1000305201231305331993070800205BA34A9D
:102F200021BAF9FC0A0A0D2050726F6772616D6D4B
:102F3000696E6720436F6D706C65746564205375AE
:102F4000636365737366756C6C79210A0D2D2D2D85
:102F50002D2D2D2D2D2D2D2D2D2D2D2D2D2D2D2DA1
:102F60002D2D2D2D2D2D2D2D2D2D2D2D2D0D0A20E1
:102F70004E616D653A20000060CD020200E8020259
:102F8000F40100006CA10202C0CD0202F4E90202C9
:102F9000A00D00001CCB02025203328052013426E5
:102FA000B803350F00010145FDAC02020345500690
:102FB000C570014013D6207001401445B000500B7D
:102FC0004202820345FFFF0F20320442083201040F
:102FD000561000010551200050074590014018424D
:102FE00004023D0545A00140194206023D07454047
:102FF00001400D8201000000FFFFFFFFFFFFFFFF08
:10300000FFFFFFFFFFFFFFFFFFFFFFFFFFFFFFFFD0
:10301000FFFFFFFFFFFFFFFFFFFFFFFFFFFFFFFFC0
:10302000FFFFFFFFFFFFFFFFFFFFFFFFFFFFFFFFB0
:10303000FFFFFFFFFFFFFFFFFFFFFFFFFFFFFFFFA0
:10304000FFFFFFFFFFFFFFFFFFFFFFFFFFFFFFFF90
:10305000FFFFFFFFFFFFFFFFFFFFFFFFFFFFFFFF80
:10306000FFFFFFFFFFFFFFFFFFFFFFFFFFFFFFFF70
:10307000FFFFFFFFFFFFFFFFFFFFFFFFFFFFFFFF60
:10308000FFFFFFFFFFFFFFFFFFFFFFFFFFFFFFFF50
:10309000FFFFFFFFFFFFFFFFFFFFFFFFFFFFFFFF40
:1030A000FFFFFFFFFFFFFFFFFFFFFFFFFFFFFFFF30
:1030B000FFFFFFFFFFFFFFFFFFFFFFFFFFFFFFFF20
:1030C000FFFFFFFFFFFFFFFFFFFFFFFFFFFFFFFF10
:1030D000FFFFFFFFFFFFFFFFFFFFFFFFFFFFFFFF00
:1030E000FFFFFFFFFFFFFFFFFFFFFFFFFFFFFFFFF0
:1030F000FFFFFFFFFFFFFFFFFFFFFFFFFFFFFFFFE0
:10310000FFFFFFFFFFFFFFFFFFFFFFFFFFFFFFFFCF
:10311000FFFFFFFFFFFFFFFFFFFFFFFFFFFFFFFFBF
:10312000FFFFFFFFFFFFFFFFFFFFFFFFFFFFFFFFAF
:10313000FFFFFFFFFFFFFFFFFFFFFFFFFFFFFFFF9F
:10314000FFFFFFFFFFFFFFFFFFFFFFFFFFFFFFFF8F
:10315000FFFFFFFFFFFFFFFFFFFFFFFFFFFFFFFF7F
:10316000FFFFFFFFFFFFFFFFFFFFFFFFFFFFFFFF6F
:10317000FFFFFFFFFFFFFFFFFFFFFFFFFFFFFFFF5F
:10318000FFFFFFFFFFFFFFFFFFFFFFFFFFFFFFFF4F
:10319000FFFFFFFFFFFFFFFFA5A54B4D0000001045
:1031A00000000002AAAA5A7F60CF020200000000BD
:1031B000020000000000000000000000000000000D
:1031C00000000000000000000000000000000000FF
:1031D0000000000000000000F8CF02020000000024
:1031E0000A56656E646F72093A204D4B53454D493E
:1031F0000A43686970093A204D4B383030300A4430
:10320000617465093A2041707220203220323032D8
:10321000350A56657273696F6E093A2056302E363C
:103220002E3200000000000000000000000000003E
:10323000403200000080000214000000180200006C
:103240000026B803004001400D000000010000000E
:04325000000000007A
:020000040000FA
:10326000A5A54B4D0000001000000002AAAA5A7F3D
:1032700060320000000000000200000000000000BA
:10328000000000000000000000000000000000003E
:10329000000000000000000000000000000000002E
:1032A000F8320000000000000A56656E646F720973
:1032B0003A204D4B53454D490A43686970093A20FD
:1032C0004D4B383030300A44617465093A204D6105
:1032D0007220323620323032350A56657273696F89
:1032E0006E093A2056302E362E32000000000000C3
:0832F0000000000000000000D6
:04000005000000C136
:00000001FF
